:040000000C94F1006B
:100004000C9400000C9400000C9400000C9400006C
:100014000C9400000C9400000C9400000C9400005C
:100024000C9400000C9400000C9400000C9400004C
:100034000C9400000C9400000C9400000C94290112
:100044000C9400000C9400000C9400000C9400002C
:100054000C943D010C9400000C9400000C940000DE
:100064000C940000041500000000000004150010AA
:100074001010100004150018181818000415001C9E
:100084001C1C1C000415001E1E1E1E000415001F4F
:100094001F1F1F000E12100C02121C000F11100E55
:1000A40001111E0001000100E8030000000000002F
:1000B400000076025452582054454136323030768E
:1000C4002E3033640020526166696E6164202D20F5
:1000D40032303136200020545258205445413632B3
:1000E4003030762E303364002020466972737420D9
:1000F400537461727420202000202020204946205F
:100104005365747570202020200044445320512EE0
:100114002047656E205365747570004946203D2064
:100124000020487A004564697420002031206B481F
:100134007A003130206B487A0031303020487A0020
:100144003530206B487A003120206B487A003130FA
:100154002020487A0031202020487A0020204B6F4C
:10016400656666205665726966792020002E004116
:100174004D20002035206B487A0035303020487AF5
:10018400005200203020202020487A002030644291
:1001940020002D3130644220002D32306442200092
:1001A4002D33306442200020202053575220000079
:1001B40080C001002D4E414E00494E460000010012
:1001C4000200A80001003103AA000C000300AC00E7
:1001D40002003B03B40101004203B6010000F8949D
:1001E400EE27EFBBF1E0F5BFE5BFF8E1A895A4B7B2
:1001F400A77FA4BFF0936000E09360008DE0A2E0CD
:10020400BB27ED938A95E9F780E098E0A0E0B1E0A0
:10021400ED930197E9F7E2ECF1E085919591009770
:1002240061F0A591B59105901590BF01F00105907D
:100234000D920197E1F7FB01F0CFE0E8EEBBEFEFA1
:10024400EDBFE8E0EEBFC0E0D3E00C94E201EA9336
:10025400FA93EFB7EA93E0910C03F0910D03319612
:10026400E0930C03F0930D03E0E0E6BDE991EFBFEA
:10027400F991E9911895EA93EFB7EA931A930A93DF
:100284000091780010917900B02EC12EF69B02C027
:10029400E5EC01C0E0ECE0937C00689420F809915F
:1002A4001991E991EFBFE99118951A930A93EA819C
:1002B400EE0FEE0FEE0FE0640E2F10E0183070F426
:1002C4000A930395EC81FD813196EC83FD8331978C
:1002D400E491EA930E942F101F5FF0CF19810881E7
:1002E40025960895E0E0E0932E03E0932F0308950C
:1002F4001A9310E0339B11E0349B1260E0912E03BB
:10030400E11711F40C94E001A0912E03A33021F421
:10031400E0912F03E11709F44BC0123031F5F09945
:1003240017C0E32DF42DA0910003B0910103809137
:10033400020390910303662777270E948912E093B2
:100344000003F093010360930203709303030BC053
:10035400E7E8F3E17E168F063CF4E72DF82DEC591F
:10036400FF4F7E2E8F2EF79A23C0F09917C0E32DEE
:10037400F42DA0910003B0910103809102039091A8
:100384000303662777270E949312A0930003B09378
:100394000103809302039093030309C0E9E7FCEE91
:1003A400E715F8052CF4E4E6F0E07E1A8F0AF79AD4
:1003B400E0912E03E0932F0310932E0319910895D7
:1003C400E0E8E0936100E0E0E0936100E5B9E0E398
:1003D400E4B9E0E0E8B9E7B9EBB9EFE0EAB9E0E0A5
:1003E400E4BDE5E0E5BDE0E0E6BDE7BDE8BDE093E2
:1003F4008000E0938100E0938500E0938400E09323
:100404008700E0938600E0938900E0938800E093FE
:100414008B00E0938A00E093B600E093B000E09391
:10042400B100E093B200E093B300E093B400E09332
:100434006900EDBBE0936800E1E0E0936E00E0E06A
:10044400E0936F00E0937000E093C100E0E8E0BF48
:10045400E0E0E0937B00E0937F00E0937E00E0EC3B
:10046400E0937C00EBE8E0937A00E0E0ECBDE093FD
:10047400BC00E0E1EA930E94A310E8E6F0E0FA93FE
:10048400EA93E0E0EA9311DFE0E7F0E0FA93EA931D
:10049400E1E0EA930ADFE8E7F0E0FA93EA93E2E0C6
:1004A400EA9303DFE0E8F0E0FA93EA93E3E0EA9307
:1004B400FCDEE8E8F0E0FA93EA93E4E0EA93F5DEA0
:1004C400E0E9F0E0FA93EA93E5E0EA93EEDEE8E9A6
:1004D400F0E0FA93EA93E6E0EA93E7DEE0EAF0E09C
:1004E400FA93EA93E7E0EA93E0DEA0E0B0E00E944A
:1004F4002913E530C1F4E0E0EA93EA930E9438104E
:10050400E8EBF0E0FA93EA930E949210E0E0EA93B9
:10051400E1E0EA930E943810E9ECF0E0FA93EA9300
:100524000E94921044C0E0E0EA93EA930E943810DB
:10053400EAEDF0E0FA93EA930E949210E0E0EA9385
:10054400E1E0EA930E943810ECEEF0E0FA93EA93CB
:100554000E949210ADE0B0E0E0EFF3EB6AE170E0EE
:100564000E943513A1E0B0E0E0EEF4E463EA70E049
:100574000E943513A9E0B0E0E0E4F9E563E777E031
:100584000E943513A9E0B0E00E9421130E94C81113
:10059400A0E0B0E080E89FE40E944412A5E0B0E04F
:1005A4000E943513A0E0B0E0E5E00E9445131A99DB
:1005B40019C0F29AE0E0EA93EA930E943810EAED57
:1005C400F0E0FA93EA930E949210E0E0EA93E1E00B
:1005D400EA930E943810EDEFF0E0FA93EA930E9458
:1005E400921001C0F298199919C0F49AE0E0EA93C4
:1005F400EA930E943810EAEDF0E0FA93EA930E943D
:100604009210E0E0EA93E1E0EA930E943810EEE011
:10061400F1E0FA93EA930E94921001C0F49862DE2A
:10062400E0917C00EE7FE0937C00E0917C00ED7F24
:10063400E0937C00E0917C00EB7FE0937C00E09110
:100644007C00E77FE0937C00E0EDF7E0FA93EA9327
:100654000E945611589A58980E944910F29BC2C0A1
:10066400F3990DC0A1E0B0E00E942113E0930003D0
:10067400F09301036093020370930303F39AF79BCF
:100684002CC00E944910E0E0EA93EA930E943810DB
:10069400EFE1F1E0FA93EA930E949210E0910003F3
:1006A400F091010360910203709103030E940A1305
:1006B400E4E1F3E0FA93EA930E94E810E4E1F3E062
:1006C400FA93EA930E948510E5E2F1E0FA93EA9343
:1006D4000E949210F798689420F820FE3AC0E0E057
:1006E400EA93E1E0EA930E943810E9E2F1E0FA9338
:1006F400EA930E949210E8EEF3E0E315F40531F476
:10070400EFE2F1E0FA93EA930E949210E0E1F7E25B
:10071400E315F40531F4E6E3F1E0FA93EA930E9479
:100724009210E4E6F0E0E315F40531F4EDE3F1E0D2
:10073400FA93EA930E949210E0E5F3ECE315F405D2
:1007440031F4E4E4F1E0FA93EA930E949210E8941D
:1007540020F8CEDD1B9927C0E32DF42DE436A0E06C
:10076400FA0719F4E8EEF3E014C0E83EA3E0FA0750
:1007740019F4E0E1F7E20DC0E031A7E2FA0719F459
:10078400E0E5F3EC06C0E035A3ECFA0761F4E4E637
:10079400F0E03E2E4F2E689420F8ECE2F1E0FA935C
:1007A400EA930E94561119991CC0E0910003F0913C
:1007B40001036091020370910303A1E0B0E00E9481
:1007C4003513F79A689420F8E8EEF3E03E2E4F2EA6
:1007D4000E944910E8EEF3E0FA93EA930E9456115E
:1007E400F2983CCFF49B1FC1F5990DC0A9E0B0E08D
:1007F4000E942113E0930003F0930103609302032A
:1008040070930303F59AF79B28C0E0E0EA93EA9318
:100814000E943810E0E2F1E0FA93EA930E94921009
:10082400E0910003F09101036091020370910303CE
:100834000E940A13E4E1F3E0FA93EA930E94E810B9
:10084400E4E1F3E0FA93EA930E948510E5E2F1E033
:10085400FA93EA930E949210F79820FE3AC0E0E0DF
:10086400EA93E1E0EA930E943810E9E2F1E0FA93B6
:10087400EA930E949210E8EEF3E0E315F40531F4F4
:10088400EBE4F1E0FA93EA930E949210E4E6F0E0DC
:10089400E315F40531F4EDE3F1E0FA93EA930E94F1
:1008A4009210EAE0F0E0E315F40531F4E2E5F1E05A
:1008B400FA93EA930E949210E1E0F0E0E315F40564
:1008C40031F4E9E5F1E0FA93EA930E949210E89496
:1008D40020F80EDD1B9927C0E32DF42DE436A0E0AB
:1008E400FA0719F4E8EEF3E014C0E83EA3E0FA07CF
:1008F40019F4E1E0F0E00DC0E130A0E0FA0719F4EA
:10090400EAE0F0E006C0EA30A0E0FA0761F4E4E6C9
:10091400F0E03E2E4F2E689420F8ECE2F1E0FA93DA
:10092400EA930E9456111A997DC0E0910003F09158
:1009340001036091020370910303A9E0B0E00E94F7
:100944003513E4E6F0E0FA93EA930E945611A9E025
:10095400B0E00E9421130E94C811A0E0B0E080E83A
:100964009FE40E944412A5E0B0E00E943513E4E63F
:10097400F0E0FA93EA930E9456110E944910E0E0D5
:10098400EA93EA930E943810E0E6F1E0FA93EA93DE
:100994000E949210A5E0B0E00E942113A0E0B0E014
:1009A40080E89FE40E944412A0E0B3E00E948F110B
:1009B4000E940513E0910003F0910103609102038A
:1009C400709103030E940A13E4E1F3E0FA93EA93BB
:1009D4000E94E810E0E0EA93E1E0EA930E94381014
:1009E400E9EFF0E0FA93EA930E949210E4E1F3E075
:1009F400FA93EA930E948510E8EBFBE0FA93EA93FA
:100A04000E945611F79A689420F8E8EEF3E03E2E1F
:100A14004F2E0E944910E8EEF3E0FA93EA930E9405
:100A24005611F498DFCEA5E0B0E00E942113E093C4
:100A34003703F09338036093390370933A03A1E0CA
:100A4400B0E00E942113E0930803F093090360933C
:100A54000A0370930B03ADE0B0E00E942113E0930E
:100A64000003F093010360930203709303037894EB
:100A7400F79B39C1E0E0EA93EA930E943810A09111
:100A84000003B09101038091020390910303E8EE07
:100A9400F3E060E070E00E94DC12E0932A03F0933C
:100AA4002B03A0910003B091010380910203909164
:100AB4000303E8EEF3E060E070E00E940113DF015D
:100AC400CB01E4E6F0E060E070E00E94DC12E09329
:100AD4002C03F0932D03E0912A03F0912B030E9441
:100AE400A8120E940A13E4E1F3E0FA93EA930E9445
:100AF400E810E0912C03F0912D030E94A8120E94AB
:100B04000A13E4E2F3E0FA93EA930E94E810E4E1C2
:100B1400F3E0FA93EA930E948510E1E7F1E0FA9397
:100B2400EA930E949210E4E2F3E0FA93EA930E94BB
:100B34008510E8EDF0E0FA93EA930E949210A091F8
:100B44002A03B0912B03A83EE3E0BE0734F4E8ED9A
:100B5400F0E0FA93EA930E949210F09935C0E3E72B
:100B6400F1E0FA93EA930E949210E8EEF3E0E315C1
:100B7400F40531F4EFE2F1E0FA93EA930E94921063
:100B8400E0E1F7E2E315F40531F4E6E3F1E0FA938A
:100B9400EA930E949210E8E8F3E1E315F40531F4D6
:100BA400E7E7F1E0FA93EA930E949210E4EFF1E0B0
:100BB400E315F40531F4EEE7F1E0FA93EA930E94C9
:100BC4009210E8ECF0E087C0E5E8F1E0FA93EA93EC
:100BD4000E949210E72DF82D0E94A8120E940A1379
:100BE400EEE0F3E0FA93EA930E94E810072C082859
:100BF40031F4E7E8F1E0FA93EA930E949210A72D0A
:100C0400B82DE0E0F0E00E94C4120E2EE7EEF3E00F
:100C14000E94B212E02191F0E8EDF0E0FA93EA9339
:100C24000E949210EEE0F3E0FA93EA930E9485109A
:100C3400E4E5F1E0FA93EA930E949210A72DB82D0F
:100C4400E8EEF3E00E94B8120E2EEFE0F7E20E9405
:100C5400B212E02191F0E8EDF0E0FA93EA930E94F9
:100C64009210EEE0F3E0FA93EA930E948510E5E235
:100C7400F1E0FA93EA930E949210A72DB82DE0E0D8
:100C8400F0E00E94BE120E2EE9E1FCEF0E94B812C1
:100C9400E02161F0EEE0F3E0FA93EA930E9485101C
:100CA400E4E5F1E0FA93EA930E949210A72DB82D9F
:100CB400E8E1FCEF0E94B2120E2EE1EFF8ED0E9483
:100CC400C412E02161F0EEE0F3E0FA93EA930E94AB
:100CD4008510E5E2F1E0FA93EA930E949210F79806
:100CE400E1E0E093310320FC02C00C94850EF699F8
:100CF4005AC4E0E0EA93E1E0EA930E9438106620E7
:100D040081F4E0E9F1E0FA93EA930E949210E7E0BB
:100D1400EA930E946410E8EDF0E0FA93EA930E94EB
:100D24009210092C0A2851F5E7E0EA93E1E0EA93EE
:100D34000E943810E0E0EA930E946410E0E0EA9335
:100D44000E946410E0E0EA930E946410E0E0EA93F9
:100D54000E946410E0E0EA930E946410E0E0EA93E9
:100D64000E946410E0E0EA930E946410E0E0EA93D9
:100D74000E946410E0E0EA930E946410EAE0E61541
:100D840081F4E0E0EA93E1E0EA930E943810E6E9B6
:100D9400F1E0FA93EA930E949210E6E0EA930E944B
:100DA4006410E4E1E61581F4E0E0EA93E1E0EA931B
:100DB4000E943810EDE9F1E0FA93EA930E94921050
:100DC400E6E0EA930E946410EEE1E61581F4E0E0C7
:100DD400EA93E1E0EA930E943810E4EAF1E0FA933E
:100DE400EA930E949210E6E0EA930E9464109B2C1E
:100DF400AC2CED2DFE2DEA57FE4FE915FA0520F532
:100E0400E5E0EA930E946410E5E0EA930E9464102E
:100E1400E5E0EA930E946410E5E0EA930E9464101E
:100E2400E5E0EA930E946410E5E0EA930E9464100E
:100E3400E5E0EA930E946410E5E0EA930E946410FE
:100E4400E5E0EA930E946410ED2DFE2DE458FE4F78
:100E5400A92DBA2D0E94D6120E2EED2DFE2DEA5785
:100E6400FE4F0E94D012E02121F1E5E0EA930E94B6
:100E74006410E5E0EA930E946410E5E0EA930E94BE
:100E84006410E5E0EA930E946410E5E0EA930E94AE
:100E94006410E5E0EA930E946410E5E0EA930E949E
:100EA4006410E5E0EA930E946410E2E0EA930E9491
:100EB4006410ED2DFE2DE859FE4FA92DBA2D0E9488
:100EC400D6120E2EED2DFE2DE458FE4F0E94D012A8
:100ED400E02121F1E5E0EA930E946410E5E0EA9361
:100EE4000E946410E5E0EA930E946410E5E0EA934E
:100EF4000E946410E5E0EA930E946410E5E0EA933E
:100F04000E946410E5E0EA930E946410E5E0EA932D
:100F14000E946410E0E0EA930E946410ED2DFE2D1F
:100F2400EC5AFE4FA92DBA2D0E94D6120E2EED2D8D
:100F3400FE2DE859FE4F0E94D012E02121F1E5E098
:100F4400EA930E946410E5E0EA930E946410E5E0ED
:100F5400EA930E946410E5E0EA930E946410E5E0DD
:100F6400EA930E946410E5E0EA930E946410E5E0CD
:100F7400EA930E946410E2E0EA930E946410E0E0C5
:100F8400EA930E946410ED2DFE2DE05CFE4FA92D26
:100F9400BA2D0E94D6120E2EED2DFE2DEC5AFE4FC8
:100FA4000E94D012E02121F1E5E0EA930E9464104E
:100FB400E5E0EA930E946410E5E0EA930E9464107D
:100FC400E5E0EA930E946410E5E0EA930E9464106D
:100FD400E5E0EA930E946410E5E0EA930E9464105D
:100FE400E0E0EA930E946410E0E0EA930E94641057
:100FF400ED2DFE2DEA5CFE4FA92DBA2D0E94D612CE
:101004000E2EED2DFE2DE05CFE4F0E94D012E0214D
:1010140021F1E5E0EA930E946410E5E0EA930E947E
:101024006410E5E0EA930E946410E5E0EA930E940C
:101034006410E5E0EA930E946410E5E0EA930E94FC
:101044006410E2E0EA930E946410E0E0EA930E94F4
:101054006410E0E0EA930E946410ED2DFE2DEE5D35
:10106400FE4FA92DBA2D0E94D6120E2EED2DFE2D67
:10107400EA5CFE4F0E94D012E02121F1E5E0EA9300
:101084000E946410E5E0EA930E946410E5E0EA93AC
:101094000E946410E5E0EA930E946410E5E0EA939C
:1010A4000E946410E5E0EA930E946410E0E0EA9391
:1010B4000E946410E0E0EA930E946410E0E0EA9386
:1010C4000E946410ED2DFE2DE25FFE4FA92DBA2D76
:1010D4000E94D6120E2EED2DFE2DEE5DFE4F0E94C7
:1010E400D012E02121F1E5E0EA930E946410E5E0EA
:1010F400EA930E946410E5E0EA930E946410E5E03C
:10110400EA930E946410E5E0EA930E946410E2E02E
:10111400EA930E946410E0E0EA930E946410E0E025
:10112400EA930E946410E0E0EA930E946410ED2DBB
:10113400FE2DE051FF4FA92DBA2D0E94D6120E2E7E
:10114400ED2DFE2DE25FFE4F0E94D012E02121F131
:10115400E5E0EA930E946410E5E0EA930E946410DB
:10116400E5E0EA930E946410E5E0EA930E946410CB
:10117400E5E0EA930E946410E0E0EA930E946410C0
:10118400E0E0EA930E946410E0E0EA930E946410B5
:10119400E0E0EA930E946410ED2DFE2DE254FF4F2F
:1011A400A92DBA2D0E94D6120E2EED2DFE2DE05142
:1011B400FF4F0E94D012E02121F1E5E0EA930E9462
:1011C4006410E5E0EA930E946410E5E0EA930E946B
:1011D4006410E5E0EA930E946410E2E0EA930E945E
:1011E4006410E0E0EA930E946410E0E0EA930E9455
:1011F4006410E0E0EA930E946410E0E0EA930E9445
:101204006410ED2DFE2DEA56FF4FA92DBA2D0E9434
:10121400D6120E2EED2DFE2DE254FF4F0E94D01259
:10122400E02121F1E5E0EA930E946410E5E0EA930D
:101234000E946410E5E0EA930E946410E5E0EA93FA
:101244000E946410E0E0EA930E946410E0E0EA93F4
:101254000E946410E0E0EA930E946410E0E0EA93E4
:101264000E946410E0E0EA930E946410ED2DFE2DCC
:10127400EC59FF4FA92DBA2D0E94D6120E2EED2D3A
:10128400FE2DEA56FF4F0E94D012E02121F1E5E045
:10129400EA930E946410E5E0EA930E946410E5E09A
:1012A400EA930E946410E2E0EA930E946410E0E092
:1012B400EA930E946410E0E0EA930E946410E0E084
:1012C400EA930E946410E0E0EA930E946410E0E074
:1012D400EA930E946410ED2DFE2DEA5BFF4FA92DC9
:1012E400BA2D0E94D6120E2EED2DFE2DEC59FF4F75
:1012F4000E94D012E02121F1E5E0EA930E946410FB
:10130400E5E0EA930E946410E5E0EA930E94641029
:10131400E0E0EA930E946410E0E0EA930E94641023
:10132400E0E0EA930E946410E0E0EA930E94641013
:10133400E0E0EA930E946410E0E0EA930E94641003
:10134400ED2DFE2DF796A92DBA2D0E94D6120E2E44
:10135400ED2DFE2DEA5BFF4F0E94D012E02121F11A
:10136400E5E0EA930E946410E5E0EA930E946410C9
:10137400E2E0EA930E946410E0E0EA930E946410C1
:10138400E0E0EA930E946410E0E0EA930E946410B3
:10139400E0E0EA930E946410E0E0EA930E946410A3
:1013A400E0E0EA930E946410ED2DFE2DB896A92D7D
:1013B400BA2D0E94D6120E2EED2DFE2DF7960E9408
:1013C400D012E02121F1E5E0EA930E946410E5E007
:1013D400EA930E946410E0E0EA930E946410E0E063
:1013E400EA930E946410E0E0EA930E946410E0E053
:1013F400EA930E946410E0E0EA930E946410E0E043
:10140400EA930E946410E0E0EA930E946410ED2DD8
:10141400FE2D7996A92DBA2D0E94D6120E2EED2DF1
:10142400FE2DB8960E94D012E02121F1E5E0EA9366
:101434000E946410E2E0EA930E946410E0E0EA9300
:101444000E946410E0E0EA930E946410E0E0EA93F2
:101454000E946410E0E0EA930E946410E0E0EA93E2
:101464000E946410E0E0EA930E946410E0E0EA93D2
:101474000E946410ED2DFE2D7196A92DBA2D0E94A7
:10148400D6120E2EED2DFE2D79960E94D012E0215B
:1014940021F1E5E0EA930E946410E0E0EA930E94FF
:1014A4006410E0E0EA930E946410E0E0EA930E9492
:1014B4006410E0E0EA930E946410E0E0EA930E9482
:1014C4006410E0E0EA930E946410E0E0EA930E9472
:1014D4006410E0E0EA930E946410ED2DFE2D3A962C
:1014E400A92DBA2D0E94D6120E2EED2DFE2D719629
:1014F4000E94D012E02121F1E3E0EA930E946410FB
:10150400E0E0EA930E946410E0E0EA930E94641031
:10151400E0E0EA930E946410E0E0EA930E94641021
:10152400E0E0EA930E946410E0E0EA930E94641011
:10153400E0E0EA930E946410E0E0EA930E94641001
:10154400ED2DFE2D3096A92DBA2D0E94CA120E2E15
:10155400ED2DFE2D3A960E94D012E02121F1E1E01A
:10156400EA930E946410E0E0EA930E946410E0E0D1
:10157400EA930E946410E0E0EA930E946410E0E0C1
:10158400EA930E946410E0E0EA930E946410E0E0B1
:10159400EA930E946410E0E0EA930E946410E0E0A1
:1015A400EA930E946410F69BA9C3E0E0EA93E1E0A9
:1015B400EA930E943810EBEAF1E0FA93EA930E946E
:1015C40092109B2CAC2CE1E4F1E0E915FA0520F52E
:1015D400E5E0EA930E946410E5E0EA930E94641057
:1015E400E5E0EA930E946410E5E0EA930E94641047
:1015F400E5E0EA930E946410E5E0EA930E94641037
:10160400E5E0EA930E946410E5E0EA930E94641026
:10161400E5E0EA930E946410A92DBA2DE2E1F1E01D
:101624000E94D6120E2EE1E4F1E00E94D012E021D5
:1016340021F1E5E0EA930E946410E5E0EA930E9458
:101644006410E5E0EA930E946410E5E0EA930E94E6
:101654006410E5E0EA930E946410E5E0EA930E94D6
:101664006410E5E0EA930E946410E5E0EA930E94C6
:101674006410E3E0EA930E946410A92DBA2DEDEE04
:10168400F0E00E94D6120E2EE2E1F1E00E94D012A8
:10169400E02121F1E5E0EA930E946410E5E0EA9399
:1016A4000E946410E5E0EA930E946410E5E0EA9386
:1016B4000E946410E5E0EA930E946410E5E0EA9376
:1016C4000E946410E5E0EA930E946410E5E0EA9366
:1016D4000E946410E0E0EA930E946410A92DBA2DE0
:1016E400EFECF0E00E94D6120E2EEDEEF0E00E9438
:1016F400D012E02121F1E5E0EA930E946410E5E0D4
:10170400EA930E946410E5E0EA930E946410E5E025
:10171400EA930E946410E5E0EA930E946410E5E015
:10172400EA930E946410E5E0EA930E946410E3E007
:10173400EA930E946410E0E0EA930E946410A92DE9
:10174400BA2DE5EBF0E00E94D6120E2EEFECF0E09D
:101754000E94D012E02121F1E5E0EA930E94641096
:10176400E5E0EA930E946410E5E0EA930E946410C5
:10177400E5E0EA930E946410E5E0EA930E946410B5
:10178400E5E0EA930E946410E5E0EA930E946410A5
:10179400E0E0EA930E946410E0E0EA930E9464109F
:1017A400A92DBA2DEFE9F0E00E94D6120E2EE5EB3A
:1017B400F0E00E94D012E02121F1E5E0EA930E94DA
:1017C4006410E5E0EA930E946410E5E0EA930E9465
:1017D4006410E5E0EA930E946410E5E0EA930E9455
:1017E4006410E5E0EA930E946410E3E0EA930E9447
:1017F4006410E0E0EA930E946410E0E0EA930E943F
:101804006410A92DBA2DECE8F0E00E94D6120E2E39
:10181400EFE9F0E00E94D012E02121F1E5E0EA9343
:101824000E946410E5E0EA930E946410E5E0EA9304
:101834000E946410E5E0EA930E946410E5E0EA93F4
:101844000E946410E5E0EA930E946410E0E0EA93E9
:101854000E946410E0E0EA930E946410E0E0EA93DE
:101864000E946410A92DBA2DEAE7F0E00E94D61276
:101874000E2EECE8F0E00E94D012E02121F1E5E028
:10188400EA930E946410E5E0EA930E946410E5E0A4
:10189400EA930E946410E5E0EA930E946410E5E094
:1018A400EA930E946410E3E0EA930E946410E0E08B
:1018B400EA930E946410E0E0EA930E946410E0E07E
:1018C400EA930E946410A92DBA2DEBE6F0E00E9481
:1018D400D6120E2EEAE7F0E00E94D012E02121F1A8
:1018E400E5E0EA930E946410E5E0EA930E94641044
:1018F400E5E0EA930E946410E5E0EA930E94641034
:10190400E5E0EA930E946410E0E0EA930E94641028
:10191400E0E0EA930E946410E0E0EA930E9464101D
:10192400E0E0EA930E946410A92DBA2DECE5F0E002
:101934000E94D6120E2EEBE6F0E00E94D012E021B7
:1019440021F1E5E0EA930E946410E5E0EA930E9445
:101954006410E5E0EA930E946410E5E0EA930E94D3
:101964006410E3E0EA930E946410E0E0EA930E94CA
:101974006410E0E0EA930E946410E0E0EA930E94BD
:101984006410E0E0EA930E946410A92DBA2DEFE4FC
:10199400F0E00E94D6120E2EECE5F0E00E94D01288
:1019A400E02121F1E5E0EA930E946410E5E0EA9386
:1019B4000E946410E5E0EA930E946410E5E0EA9373
:1019C4000E946410E0E0EA930E946410E0E0EA936D
:1019D4000E946410E0E0EA930E946410E0E0EA935D
:1019E4000E946410E0E0EA930E946410A92DBA2DCD
:1019F400E3E4F0E00E94D6120E2EEFE4F0E00E9441
:101A0400D012E02121F1E5E0EA930E946410E5E0C0
:101A1400EA930E946410E5E0EA930E946410E3E014
:101A2400EA930E946410E0E0EA930E946410E0E00C
:101A3400EA930E946410E0E0EA930E946410E0E0FC
:101A4400EA930E946410E0E0EA930E946410A92DD6
:101A5400BA2DE8E3F0E00E94D6120E2EE3E4F0E0A3
:101A64000E94D012E02121F1E5E0EA930E94641083
:101A7400E5E0EA930E946410E5E0EA930E946410B2
:101A8400E0E0EA930E946410E0E0EA930E946410AC
:101A9400E0E0EA930E946410E0E0EA930E9464109C
:101AA400E0E0EA930E946410E0E0EA930E9464108C
:101AB400A92DBA2DEDE2F0E00E94D6120E2EE8E335
:101AC400F0E00E94D012E02121F1E5E0EA930E94C7
:101AD4006410E5E0EA930E946410E3E0EA930E9454
:101AE4006410E0E0EA930E946410E0E0EA930E944C
:101AF4006410E0E0EA930E946410E0E0EA930E943C
:101B04006410E0E0EA930E946410E0E0EA930E942B
:101B14006410A92DBA2DE3E2F0E00E94D6120E2E35
:101B2400EDE2F0E00E94D012E02121F1E5E0EA9339
:101B34000E946410E5E0EA930E946410E0E0EA93F6
:101B44000E946410E0E0EA930E946410E0E0EA93EB
:101B54000E946410E0E0EA930E946410E0E0EA93DB
:101B64000E946410E0E0EA930E946410E0E0EA93CB
:101B74000E946410A92DBA2DE9E1F0E00E94D6126A
:101B84000E2EE3E2F0E00E94D012E02121F1E5E024
:101B9400EA930E946410E3E0EA930E946410E0E098
:101BA400EA930E946410E0E0EA930E946410E0E08B
:101BB400EA930E946410E0E0EA930E946410E0E07B
:101BC400EA930E946410E0E0EA930E946410E0E06B
:101BD400EA930E946410A92DBA2DE1E1F0E00E947D
:101BE400D6120E2EE9E1F0E00E94D012E02121F19C
:101BF400E5E0EA930E946410E0E0EA930E94641036
:101C0400E0E0EA930E946410E0E0EA930E9464102A
:101C1400E0E0EA930E946410E0E0EA930E9464101A
:101C2400E0E0EA930E946410E0E0EA930E9464100A
:101C3400E0E0EA930E946410A92DBA2DEAE0F0E0F6
:101C44000E94D6120E2EE1E1F0E00E94D012E021B3
:101C540021F1E3E0EA930E946410E0E0EA930E9439
:101C64006410E0E0EA930E946410E0E0EA930E94CA
:101C74006410E0E0EA930E946410E0E0EA930E94BA
:101C84006410E0E0EA930E946410E0E0EA930E94AA
:101C94006410E0E0EA930E946410A92DBA2DE0E0FC
:101CA400F0E00E94CA120E2EEAE0F0E00E94D01288
:101CB400E02121F1E2E0EA930E946410E0E0EA937B
:101CC4000E946410E0E0EA930E946410E0E0EA936A
:101CD4000E946410E0E0EA930E946410E0E0EA935A
:101CE4000E946410E0E0EA930E946410E0E0EA934A
:101CF4000E946410E0E0EA930E946410E89420F8E3
:101D0400E1E0E09331030E947A01A0910C03B091C9
:101D14000D031B9754F0E0917A00E064E0937A009D
:101D2400E0E0E0930C03E0930D031B9926C0E32D40
:101D3400F42DE43FA1E0FA0719F4E8EEF3E014C04F
:101D4400E83EA3E0FA0719F4E8E8F3E10DC0E83847
:101D5400A3E1FA0719F4E0E1F7E206C0E031A7E2F3
:101D6400FA0759F4E4EFF1E03E2E4F2EF79AECE235
:101D7400F1E0FA93EA930E94561119992FC0E62DC7
:101D8400F0E0309739F4EAE06E2E689420F82C984D
:101D94002D9A1EC0EA30A0E0FA0731F4E4E16E2E79
:101DA400689420F82C9A13C0E431A0E0FA0739F4BF
:101DB400EEE16E2E689420F82C9A2D9A09C0EE312B
:101DC400A0E0FA0759F46624689420F82C982D981A
:101DD400ECE2F1E0FA93EA930E9456111A9918C0C2
:101DE400E0E0F099E1E0E03019F4F09AF79A06C0E7
:101DF400E13071F4F098F79A77248824ECE2F1E06A
:101E0400FA93EA930E9456110E944910689420F8AC
:101E1400A0E03299A1E0E0E0F199E1E0B0E0A7FDB3
:101E2400BFEFF0E0EA17FB0741F1F1990EC0E0E1E2
:101E3400FAE86EE270E0E0930003F093010360932C
:101E4400020370930303F19A0DC0E0EFF3EB6AE130
:101E540070E0E0930003F093010360930203709336
:101E64000303F198F79AECE2F1E0FA93EA930E9403
:101E740056110E944910689420F8E0E0319BE1E09B
:101E84000E2EA0E0F699A1E0E0E00E94AD12E02160
:101E940019F0F69A689420F8E0E03199E1E00E2E0A
:101EA400A0E0F699A1E0E1E00E94AD12E02119F072
:101EB400F698689420F8A0E01A9BA1E0E0E01B9B50
:101EC400E1E0EA23C9F0F894E0910003F091010302
:101ED4006091020370910303ADE0B0E00E943513FA
:101EE4000E944910E8EEF3E0FA93EA930E94561137
:101EF400F79A689420F87894A0913103A13011F0F6
:101F04000C94FB0FF894F69B09C0E0910003F09148
:101F14000103609102037091030318C0E091080368
:101F2400F091090360910A0370910B03A0910003DF
:101F3400B091010380910203909103030E948E12D9
:101F4400E72DF82D0E94A8120E948912E093040341
:101F5400F09305036093060370930703E0E0E093B6
:101F64003603E0913703F09138036091390370919F
:101F74003A03A0910403B091050380910603909164
:101F840007030E9411130E94F611A2E3B3E00E941A
:101F94008F110E9405135A9A5A98E0E0E093300397
:101FA400A0913003A530E8F45524E8E05E1698F4D7
:101FB400E0913003F0E0EE5CFC4F1080E52DA1E0F1
:101FC4000E94A012E12111F4599801C0599A5B9A18
:101FD4005B985394EACFE0913003EF5FE0933003D2
:101FE400DFCF59985A9A5A98E0E0E09331037894F5
:101FF40083CF0C943A05FFCFE881E07111F05D9A2C
:1020040001C05D98E881E07211F02F9A01C02F9809
:10201400E881E07411F02E9A01C02E98E881E078EE
:1020240011F05C9A01C05C9885E08A95F1F75E9A9C
:102034008DE08A95F1F75E988DE08A95F1F7C4C03A
:10204400E881EA93D9DFE881E295E883E881EA93BD
:10205400D3DF85E88A95F1F7B7C0E981EA93F0DF29
:10206400289AE881EA93ECDF28980FC0E881F0E031
:10207400E55CFC4FE081A981EA0FEA93E1DFE981A5
:10208400E0933F03E881E093400322960895E2E061
:10209400EA93D6DFE3E0F0E0FA93EA930E94561164
:1020A400ECE0EA93CDDFE1E0EA93CADFE3E0F0E0BD
:1020B400FA93EA930E945611E0E0E0934003E09320
:1020C4003F030895A881AA3031F0E0914103A09123
:1020D4003F03AE1768F0E0E0EA93E0914003EF5F5E
:1020E400E0934003EA93C2DFA881AA3009F46CC0EC
:1020F400E0913F03EF5FE0933F03289AE881EA937E
:102104009FDF289861C01A93A981BA81ED91A983B0
:10211400BA831E2FE03019F01A93D4DFF5CF0EC026
:102124001A93E981FA813196E983FA833197E4912C
:102134001E2FE03019F01A93C5DFF3CF18812396D0
:102144000895559A279A269A549A569A209A579AF5
:102154005E9828985F98E881E0934103E058E09303
:102164003D03E881E054E0933E03E4E1F0E0FA93B8
:10217400EA930E945611E0E3EA933EDF88EC90E094
:102184000197F1F7E0E3EA9337DF88EC90E00197F9
:10219400F1F7E0E3EA9330DF88EC90E00197F1F7A0
:1021A400E0E2EA9329DF88EC90E00197F1F7E8E2B6
:1021B400EA9346DFE4E0EA9343DFE5E8EA9340DFAD
:1021C400E6E0EA933DDF63DF2196089524971A93AE
:1021D4000A93E0E0FAEC6AE97BE3EA83FB836C832D
:1021E4007D8300E0AB85AA2392F4E885F9856A85AE
:1021F4007B850E949812E887F9876A877B87AE817E
:10220400BF811196AE83BF831197EDE2EC93EA810F
:10221400FB816C817D81A885B9858A859B850E9417
:10222400DC121E2F103071F4003061F4AA81BB81DE
:102234008C819D81A130E0E0BE07E0E08E07E0E004
:102244009E0751F4AE81BF811196AE83BF8311976F
:10225400E12FE05DEC9301E0EA81FB816C817D81FB
:10226400A885B9858A859B850E940113E887F9872B
:102274006A877B87AA81BB818C819D81EAE0F0E03B
:1022840060E070E00E94DC12EA83FB836C837D8350
:102294000E94561309F0BBCFAE81BF81E0E0EC93FE
:1022A400198108812C960895E991F991309639F0B5
:1022B40080ED97E00197F1F7A8953197C9F7089554
:1022C400552342F4503811F4E0FF04C03196691FDD
:1022D400791F6BF050E8572711F45F9373C05F3F89
:1022E40031F0660F000C57956795752F08955F932D
:1022F40000200AF073C06CC050E8192E1522880F14
:10230400991F9527550F879550E8072E0522660FCC
:10231400771F7527550F67950895689401C0E89451
:102324005F93F2DF703818F07F3F08F44BC056E13A
:10233400571BAAF4519558300EF4593030F0EFEF92
:10234400FFEF6FEF7FE777F91AC077275523B9F0CE
:10235400EE0FFF1F661F771F5A95D1F710C077271E
:10236400583028F0EF2FF62F672F5850F9CF552308
:1023740031F076956795F795E7955A95D1F7002052
:102384000AF4D4D05F910895689401C0E89430971A
:1023940060407040B1F0002426F0772312F40094DA
:1023A400C5D0172E7EE1112032F07A95EE0FFF1F73
:1023B400661F111CF9CFEF2FF62F612D5F938ADF73
:1023C4005F910895EE27FF27662777275F91089589
:1023D400EFEFFFEF6FE77FEF5F910895EFEFFFEF10
:1023E4006FE77FE75F9108955F9386DF703851F35D
:1023F400903841F301240894791F23F41CF300203E
:102404003AF3ECCF0F921F932F933F934F931127DF
:1024140022279927689FA0018F9F302D410D591FB6
:102424006B9F300D411D591F8E9F27D0BF9F25D014
:102434006A9F23D0BE9F1DD0AF9F1BD0AE9F110DAE
:10244400291F391F491F591FE32FF42F652F522FBE
:102454004F913F912F911F910F9066232AF0550FB2
:10246400EE1FFF1F661F02C073954BF229DF5F91B9
:102474000895100D211D391F02C0200D311D491F63
:10248400591F08955F9338DF703821F411200AF43E
:102494009FCFA4CF903809F495CF01240894970BCB
:1024A4001BF4D4F30020F3CF792F1F932F933F9382
:1024B4004F9311241127222733274427552790E2CD
:1024C400AE17BF078607410730F0AE1BBF0B860B64
:1024D400410B089401C08894551F221F331F111CFF
:1024E400AA1FBB1F881F441F9A9551F7F901612D3C
:1024F4004F913F912F911F91662332F0550FEE1F9C
:10250400FF1F661F7A9543F2DBDE5F910895EA0FA1
:10251400FB1F681F791F0895AE0FBF1F861F971FEB
:102524000895AE1BBF0B860B970B0895F09560952D
:102534007095E195FF4F6F4F7F4F0895EE230E2E58
:10254400EA2F19F0EE0F0A94E9F708956F2F660F3A
:10255400660B762F0895EA17E1E009F0EE27089557
:10256400EA17FB07E1E00CF4EE270895AE17BF0766
:10257400E1E00CF4EE270895AE17BF07E1E00CF09C
:10258400EE270895EA17FB07E1E00CF0EE27089523
:10259400AE17BF07E1E008F4EE270895AE17BF07B2
:1025A400E1E008F0EE270895EA17FB07E1E008F000
:1025B400EE2708953F934F935F93002411244427FB
:1025C400552730E2AA0FBB1F881F991F001C111C3E
:1025D400441F551F0E1A1F0A460B570B28F40E0EE4
:1025E4001F1E461F571F01C0A1603A9559F7FD01F0
:1025F400BC01D001CA015F914F913F910895DADF88
:10260400FD01BC010895ED93FD936D937C930895B2
:102614007A936A93FA93EA930895689401C0E894CC
:1026240001D0B5DE182E862F612D192E972F712D0E
:102634001B2EBF2FF12D1A2EAE2FE12D08951296C9
:1026440002D0BF011297119602D0FE2F1197F9996B
:10265400FECFFF93FFB7F894A1BDB2BDF89AE0B5E1
:10266400FFBFFF91089507D012960F01FB0103D01D
:10267400F0011297089507D01196EF93EF2F03D02E
:10268400EF9111970895F99B02C0A895FCCF9FB7CD
:10269400F894A1BDB2BDF89A80B5E81719F0E0BD71
:1026A400FA9AF99A9FBF0895309760407040089550
:00000001FF
